:020000020000FC
:1000000012C0189518951895189518951895189563
:100010001895189518951FC0189518951895189546
:1000200018951895189500271FEFEFEFE8BBE1BB77
:10003000EFEDEDBFE0E2E5BFE0E8E8B9C0E6D0E013
:10004000E1E6E993ECEDE993E0E2EBBFEFE1E0BD3F
:1000500078948895FECFE0E0B09BE0EAB19BE0E2C7
:10006000B29BE0ECB39BE0E4B49BE0E8EE2361F0EC
:10007000C2E6D0E0E993E095E99307D066D0E6B315
:10008000EF3F11F02AD0FACF18953DD03CD03BD0AD
:100090003AD039D038D037D036D035D034D033D02C
:1000A00032D031D030D02FD02ED04BD04AD049D002
:1000B00048D047D046D045D044D0C0E6D0E023D089
:1000C000E991F8E03ED0EE0F10F43BD03AD01BD0CF
:1000D000FA95C1F7C436A1F7089515D014D013D0FE
:1000E00012D011D010D00FD00ED00DD00CD00BD01C
:1000F0000AD009D008D007D006D023D022D021D0F2
:1001000020D001D00895A7E012BB17D00000000056
:1001100002BB13D00000000012BB0FD00000000093
:1001200002BB0BD00000000012BB07D00000000093
:1001300002BB03D0AA9541F708950000000000001B
:100140000895A8EBAA95F1F70895BFEBFADFBA95E9
:04015000E9F708952E
:00000001FF
